:100000000C941E060C94DC270C9409280C944606CC
:100010000C94E8120C9446060C9446060C94460682
:100020000C9446060C9446060C9446060C94460620
:100030000C9446060C9446060C9446060C94460610
:100040000C9436280C9446060C94072C0C944A2CDD
:100050000C9446060C9446060C9446060C944606F0
:100060000C9446060C9446066D18CF18AE18B118BD
:10007000B418B718BA18BD18C018CF18C918011A83
:10008000031A031A011A031A031A031A031A031A8A
:10009000031A031A031A031A031A031A031A031A78
:1000A0008719031A031A031A031A031AF818031AF2
:1000B000031A031A031A031A031A031A031A031A58
:1000C000031A031A031A031A031A031A931993192A
:1000D0009319931993199319931993199319031A4F
:1000E000031A031A031A031A031AF8189219921919
:1000F00092199219031AA019A619AC19B219B819B4
:10010000BE19C419CA19D419DE19E819F219391916
:10011000FB18031A031A031A031A8719031A031A7E
:10012000031A031A031A031A031A031A91199119CD
:1001300091199119031AA019A619AC19B219B81975
:10014000BE19C419CA19D419DE19E819F2193919D6
:10015000FB18031A031A031A031A8719361A361AD8
:10016000361A361A361A361A361A361A361A361A0F
:10017000361A361A361A4D1B4D1B4D1B4D1B4D1B87
:100180004D1B7B1A851A8F1A991AF71A011B101B1F
:10019000211BA91CBE1CCA1CD31CE21C071D101D60
:1001A000591D221D6B20712077207E208C20AE20CF
:1001B000CC20456E746572206D656E752E2E2E00F6
:1001C000546F67676C6564206D6963726F50504D42
:1001D00000546F67676C656420696E76657274653C
:1001E000642050504D2100546F67676C6564205443
:1001F00058206D7574696E672100546F67676C6570
:10020000642074656C656D65747279210050726F3D
:10021000746F636F6C206572726F72207769746897
:100220002052580054696D656F7574207768656E4B
:1002300020636F6E6E656374696E6720746F205201
:100240005800507265737320616E79206B65792058
:10025000746F2063616E63656C00436F6E6E6563DF
:1002600074696E6720746F2052582C20706F776508
:100270007220757020746865205258202877697440
:10028000682062696E6420706C7567206966206EF4
:100290006F74207573696E6720616C776179732064
:1002A00062696E642900546F67676C656420276912
:1002B0006D6D656469617465206F75747075742700
:1002C00000546F67676C65642027736C61766520E6
:1002D0006D6F64652700546F67676C6564202761E4
:1002E0006C776179732062696E642700546F676769
:1002F0006C65642050504D206368616E6E656C20A3
:100300006C696D69740053657420525353492069B8
:100310006E6A656374696F6E206368616E6E656C8A
:100320002028303D3D64697361626C652900536526
:10033000742050504D206D696E696D756D20737914
:100340006E630053657420626561636F6E20696E31
:1003500074657276616C0053657420626561636FC9
:100360006E2064656C617900536574206265616319
:100370006F6E206672657175656E637920696E2097
:10038000487A3A20303D64697361626C652C205074
:10039000783D504D52206368616E6E656C20782CFC
:1003A0002046783D465253206368616E6E656C202E
:1003B00078005365742050574D2073746F7020641B
:1003C000656C61792028302064697361626C6564B2
:1003D0002C20312D323535203D3D20302E317320FB
:1003E0002D2035306D696E29005365742050504DB5
:1003F0002073746F702064656C61792028302064EC
:10040000697361626C65642C20312D323535203D75
:100410003D20302E3173202D2035306D696E29003E
:10042000536574206661696C736166652064656CF0
:1004300061792028302064697361626C65642C20C6
:10044000312D323535203D3D20302E3173202D2089
:1004500035306D696E29002A2A2A2A2A2A2A2A2A50
:100460002A2A2A2A2A2A2A2A2A2A2A2A2A2A2A2AEC
:100470002A2A2A2A0052582041636B6564202D20C5
:1004800072657665727420737563636573736675E0
:100490006C21002A2A2A2A2A2A2A2A2A2A2A2A2AAD
:1004A0002A2A2A2A2A2A2A2A2A2A2A2A2A2A2A2AAC
:1004B000002A2A2A2A2A2A2A2A2A2A2A2A2A2A2AC6
:1004C0002A2A2A2A2A2A2A2A2A2A2A2A2A2A00528E
:1004D000582041636B6564202D20757064617465DC
:1004E000207375636365737366756C21002A2A2A0D
:1004F0002A2A2A2A2A2A2A2A2A2A2A2A2A2A2A2A5C
:100500002A2A2A2A2A2A2A2A2A2A0056616C696457
:100510002063686F69636573206172653A205B319F
:100520005D2D5B31365D20286368616E6E656C20E1
:10053000312D31362900536574206F7574707574D0
:1005400020666F7220706F727420005B585D2061AE
:10055000626F7274206368616E67657320616E6498
:10056000206578697420525820636F6E6669670051
:100570005B535D20736176652073657474696E6783
:100580007320746F205258005B525D20726576654F
:1005900072742052582073657474696E6773207486
:1005A0006F2064656661756C747300557365206EA9
:1005B000756D62657273205B312D445D20746F2010
:1005C0006564697420706F727473205B452D515D92
:1005D00020666F722073657474696E677300202DD6
:1005E00020726563656976657220636F6E66696700
:1005F000757261746F722C20727820737720000AF4
:100600000A6F70656E4C52536E67200053657420FC
:1006100073657269616C2062617564726174653AB8
:10062000200056616C69642063686F696365733A82
:100630002031202D20342B34202F2032202D203823
:10064000202F2033202D20382B34202F2034202D14
:10065000203132202F2035202D2031322B34202FF5
:100660002036202D20313600536574204368616E9A
:100670006E656C20636F6E6669673A20005365741F
:100680002044617461726174652028302D32293AEA
:10069000200053657420486F70206368616E6E653A
:1006A0006C7320286D61782032342C207365706162
:1006B000726174656420627920636F6D6D61732966
:1006C0002076616C69642076616C75657320312DCC
:1006D0003235353A2000536574206368616E6E656B
:1006E0006C2073706163696E6720287831306B48C5
:1006F0007A293A200053657420524620706F77653E
:10070000722028302D37293A200053657420524634
:10071000206D6167696320286865782920652E67E8
:100720002E20307844454144463030443A2000532E
:1007300065742062617365206672657175656E63AC
:10074000792028696E20487A293A20005B5A5D207A
:10075000656E746572207265636569766572206383
:100760006F6E66696775726174696F6E2075746902
:100770006C79005B465D20646973706C61792061FF
:10078000637475616C206672657175656E63696509
:10079000732075736564005B525D2063616C6375E3
:1007A0006C6174652072616E646F6D206B65792079
:1007B000616E6420686F70206C697374005B495DC2
:1007C000207265696E697469616C697A6520736508
:1007D0007474696E677320746F20736B65746368DB
:1007E0002064656661756C7473005B585D2072658A
:1007F00076657274206368616E67657320616E64EC
:100800002065786974206D656E75005B535D20739B
:100810006176652073657474696E677320746F20E8
:10082000454550524F4D20616E64206578697420B3
:100830006D656E7500557365206E756D62657273BA
:10084000205B302D395D20746F20656469742070E1
:100850006172616D657465727300202D2053797328
:1008600074656D20636F6E66696775726174696F18
:100870006E000A0A6F70656E4C52536E672000510D
:1008800029204F7574707574206265666F726520DB
:100890006C696E6B20283D465329203A2000502970
:1008A00020536C617665206D6F64652028657870D3
:1008B0006572696D656E74616C293A20004F29205C
:1008C00054696D65642042494E44206174207374FC
:1008D000617274757020203A20004E292050504DCE
:1008E000206F7574707574206C696D69746564200F
:1008F000202020203A200044495341424C454400E6
:100900004D292050504D205253534920746F20637D
:1009100068616E6E656C202020203A20004C2920F2
:1009200050504D206D696E696D756D2073796E63E1
:10093000202875732920203A200044495341424C15
:100940004544004B29204661696C736166652062ED
:100950006561636F6E20696E74762E2028312D32AA
:10096000353573293A20004A29204661696C736144
:10097000666520626561636F6E2064656C617920D5
:1009800028302D323535203D3E20313073202D204A
:100990003135306D696E293A200049292046616958
:1009A0006C7361666520626561636F6E206672714B
:1009B0002E203A200048292050574D2073746F7024
:1009C0002064656C6179202020202020203A2000BE
:1009D00047292050504D2073746F702064656C61FE
:1009E00079202020202020203A200046292046611E
:1009F000696C736166652064656C617920202020D4
:100A00002020203A200050574D206368616E6E65AB
:100A10006C200066756E6374696F6E3A2000292041
:100A2000706F72742000506F776572546F776572C3
:100A300000445446205548462033322D62697420C4
:100A400031306368004F70656E4C52536E67525878
:100A5000206D696E6920342F36636800466C7974A6
:100A6000726F6E2F4F72616E6765525820554846FF
:100A70002038636800525820747970653A20004429
:100A8000697361626C656400487A00203D3D200016
:100A900043616C63756C61746564207061636B6540
:100AA0007420696E74657276616C3A200042292068
:100AB0004D6963726F202868616C66292050504D23
:100AC000202020203A00412920496E766572746505
:100AD000642050504D20696E20202020203A0030A4
:100AE00029204D7574652062757A7A657220286DAB
:100AF0006F73746C79293A003929205365726961E2
:100B00006C2062617564726174653A00736D617224
:100B100074506F7274004672536B79005472616E38
:100B200073706172656E740044697361626C6564B0
:100B30000038292054656C656D657472793A2020FF
:100B40002020202020003729204368616E6E656CCC
:100B500020636F6E6669673A202000362920446161
:100B60007461726174652028302D32293A2020206A
:100B700000352920486F70206368616E6E656C7364
:100B80003A2020202020003429204368616E6E65C1
:100B90006C2073706163696E673A202000332920EE
:100BA000524620706F7765722028302D37293A2001
:100BB0002020003229205246206D616769633A2067
:100BC0002020202020202020003129204261736530
:100BD000206672657175656E63793A202020000089
:100BE00000000700020100000304060000000000EE
:100BF00000000001020408102040800102040810D7
:100C00002001020408102004040404040404040263
:100C10000202020202030303030303000000002395
:100C2000002600290000000000250028002B0000FD
:100C3000000000240027002A0000382D11241FBEC8
:100C4000CFEFD8E0DEBFCDBF13E0A0E0B1E0EEE72C
:100C5000F0E602C005900D92A83CB107D9F716E066
:100C6000A8ECB3E001C01D92AC38B107E1F71CE07D
:100C7000CCE3DCE004C02297FE010E94412ECA337F
:100C8000D107C9F70E94742D0C943D300C940000DC
:100C900080917105813019F482E080937105809113
:100CA0007105833019F484E0809371050895A89547
:100CB0000895DC01ED91FC910190F081E02D099502
:100CC00008952091720530917305382748E0C901D5
:100CD000880F991F37FF06C09C0151E2252750E17C
:100CE000352701C09C01415091F730937305209343
:100CF0007205089588E38093740580E092ECA1E08A
:100D0000B0E08093750590937605A0937705B09336
:100D1000780587E08093810580EC92E9ADEEB9E13A
:100D20008093790590937A05A0937B05B0937C0519
:100D300085E0809382058DEE9EEFADEABEED809357
:100D40007D0590937E05A0937F05B0938005E3E831
:100D5000F5E080E090E0863028F4DC01AF54BC4F31
:100D60002C9101C020E0219301968831910599F7DB
:100D700082E080939B058AE080939C05089580EC37
:100D800091EDA8E9BBE18093B9059093BA05A093D2
:100D9000BB05B093BC0580E090E0A0E0B0E5809397
:100DA000BD059093BE05A093BF05B093C005E1ECCF
:100DB000F5E080E081938F5F8031E1F70895A0E056
:100DC000B0E0E5EEF6E00C940A2ED82F0E948C28B5
:100DD0006115710581059105C9F30E94AD2E109230
:100DE0007D0510927E0510927F0510928005C4E06B
:100DF000812C912C54018A94C0907D05D0907E0561
:100E0000E0907F05F0908005FE2CED2CDC2CCC24AE
:100E10000E94A82EA50194010E94E92D6C0D7D1D54
:100E20008E1D9F1D60937D0570937E0580937F05C9
:100E300090938005C15001F7DD2309F450C003E809
:100E400015E0E801A12CB12C62E3C62ED12CE12CD7
:100E5000F12C8881882309F442C0B39419F40E94CC
:100E60007A063DC00E94A82EA70196010E94E92D96
:100E7000E1E0E60FA3E8B5E08A2F801B8A1520F495
:100E80008D918E13F9CFE9CF2091820530E0A0E15A
:100E9000B7E20E94812D9B01AC01AE2FB0E00E9411
:100EA000902D4090790550907A0560907B05709068
:100EB0007C05640D751D861D971D4090B9055090E9
:100EC000BA056090BB057090BC05461657066806CB
:100ED000790618F2E993A39488E1A812BACFCDB7A6
:100EE000DEB7E0E10C94262E8436910520F4BC0197
:100EF00080E090E017C09C018E3B910528F42A55B4
:100F00003109AAE0B0E00CC0823D910528F4245BD1
:100F10003109A4E6B0E004C02D5C3109A8E5B2E0D7
:100F20000E94812DA4E6B0E09B01AC010E94902DAF
:100F3000089590E08C599F4F0E947407089561E0D6
:100F400089E00E94392960E089E00E9472290895B1
:100F5000892B11F061E001C060E089E00E947229F4
:100F6000089560E08EE00E94392961E08FE00E94E0
:100F7000392961E082E00E94392960E083E00E9423
:100F8000392961E084E00E943929089542E050E067
:100F900068E476E081E00E94BC270895E3E0F0E099
:100FA00089E080935700E491E67081E0E63009F033
:100FB00080E00895CF93DF93C82F0E94CE07882347
:100FC00081F0DFB781E080937005F8940E945706A6
:100FD00088E180936000C0936000C1110E945706B1
:100FE000DFBFDF91CF9108958F929F92AF92BF9212
:100FF000CF92DF92EF92FF92CF93FC01C0A5EC2F2E
:10100000E770F0E0E758FC4FA081B0E0C7FF03C0F5
:1010100024E130E002C02FE030E0FC0197A183E141
:10102000989FF0011124E25CFE4F80809180A280A5
:10103000B380A20FB31F20E43FE14DE750E00E94D0
:101040009B2DA50194010E94C72D8C2F887149F416
:1010500069017A01E0EDCE0EE7E0DE1EE11CF11C35
:101060001BC0C7FF05C060E47AE88CE29EE004C0C4
:1010700060E07EEE8AEB9BE069017A01F8EBCF0E2F
:10108000FBE0DF1EE11CF11CA50194010E94C72DAD
:10109000C20ED31EE41EF51EC701B60169517C4F76
:1010A0008F4F9F4F28EE33E040E050E00E94C72D65
:1010B000A8EEB3E00E94902DCF91FF90EF90DF90CB
:1010C000CF90BF90AF909F908F9008958F3F9105E4
:1010D00051F048F0811522E0920738F081159340D5
:1010E00030F482E0089580E0089581E0089583E07F
:1010F0000895A0E0B0E0EFE7F8E00C94132EEB01C8
:101100008A01B82FB695A0E028813981F8012083A3
:101110002A813B8121832C813D8122832E813F8145
:101120002383688179814A815B812C813D81EE81B5
:10113000FF819F2F9295990F990F907C272F2370F5
:10114000922B252F2370220F220F922B232F2370F7
:101150002295207F922BF80194830B5F1F4F2896D6
:10116000AF5FBA1788F680FF24C0888199810E94FA
:101170006608D82E8A819B810E946608E82E8C81A1
:101180009D810E946608F82E8E819F810E946608CC
:10119000F0E4DF9EA001112490E1E99E900111246A
:1011A000242B282BE4E0FE9EB0011124262BF8010D
:1011B0002083CDB7DEB7E7E00C942F2E803223E0FA
:1011C000920708F1883E23E0920740F48F51934044
:1011D000E4E096958795EA95E1F70895803D27E04C
:1011E000920718F48C5D93400895883928E092079F
:1011F00068F4885C974074E0969587957A95E1F756
:101200008D509C4F089580E090E008958FEF93E01B
:1012100008958C30910540F4A4E0880F991FAA9599
:10122000E1F7885D9C4F0895843F23E0920718F40E
:1012300084529C4F0895811524E0920740F486570C
:10124000934FF4E0880F991FFA95E1F7089580E92C
:1012500098E008959C013695279525753575821B74
:10126000930B9C0123733373969587959695879579
:1012700083739373820F931F9C0154E036952795D7
:101280005A95E1F7280F391F2F703F7041E051E068
:10129000249FC001259F900D349F900D1124892F0C
:1012A00008955A98882319F00000419A02C000005E
:1012B000419800005A9A000008955A9A000086B199
:1012C0005A98000081700895CF93DF93D82F5C9ACD
:1012D0005A985C98C8E08D2F80780E945109DD0FE4
:1012E000C150C9F75A98DF91CF9108958F770E9426
:1012F00064090895CF93DF93D82FC8E08D2F8078AD
:101300000E945109DD0FC150C9F75A98DF91CF9162
:101310000895CF93DF935A98C8E080E0D82FDD0F6F
:101320000E945D098D0FC150C9F7DF91CF910895DB
:101330000E9476090E9489095C9A0895A1E0B0E0B4
:10134000E4EAF9E00C94182E806869830E9464092D
:101350006981862F0E947A095C9A2196E2E00C94BA
:10136000342ECF93C0917D05C827E82FF0E0EC58CC
:10137000FA4F678589E70E949E096C2F8DE30E94D2
:101380009E096C2F82E40E949E09CF91089586E207
:101390000E9498090895CF93DF93EC016C818CE152
:1013A0000E949E096D818DE10E949E096E818EE1F1
:1013B0000E949E096F8180E20E949E09688581E2F9
:1013C0000E949E09698582E20E949E096A8583E2E5
:1013D0000E949E096B8584E20E949E096C8585E2CD
:1013E0000E949E096D858AE20E949E096E858EE6A6
:1013F0000E949E096F858FE60E949E09688980E79A
:101400000E949E09698981E70E949E096A8982E794
:101410000E949E09DF91CF910895CF92DF92EF92C3
:10142000FF92CF93DF936B017C01C11488E3D80650
:101430008CE9E8068CE1F80628F5C701B60120E83A
:1014400036E948E950E00E94C72DE901689760E855
:1014500079E687E69FEF0E94A32D6C0D7D1D8E1D02
:101460009F1DF2E0660F771F881F991FFA95D1F72D
:1014700021E732E040E050E00E94C72DF22EE32E3B
:1014800080E421C0C701B60120E03DE241E351E024
:101490000E94C72DE901689760E073ED8EEC9EEF26
:1014A0000E94A32D6C0D7D1D8E1D9F1D660F771F45
:1014B000881F991F21E732E040E050E00E94C72DCD
:1014C000F22EE32E80E66C2F6F71680F85E70E9485
:1014D0009E096E2D86E70E949E096F2D87E70E9468
:1014E0009E09DF91CF91FF90EF90DF90CF9008950C
:1014F000682F8DE60E949E0908958F929F92AF9269
:10150000BF92CF92DF92EF92FF92CF93DF93D82FCB
:1015100083E00E94980980936F0584E00E949809F7
:1015200080936E0560E086E00E949E0961E087E09E
:101530000E949E096FE789E00E949E0965E08AE0AB
:101540000E949E0962E18BE00E949E0965E18CE0A9
:101550000E949E096DEF8DE00E949E0960E08EE082
:101560000E949E09DD2319F08BE291E008C02091D2
:101570009B0533E1239FC0011124825C9E4F0E9492
:10158000CB096CE880E30E949E096FE082E30E9431
:101590009E0962E483E30E949E0980919C0587FF77
:1015A00002C064E101C06AE084E30E949E096AE22D
:1015B00085E30E949E096DE286E30E949E0964ED28
:1015C00087E30E949E0960E088E30E949E0960E034
:1015D00089E30E949E09D11109C0C0907D05D09079
:1015E0007E05E0907F05F090800507C0C5E9CC2E10
:1015F000C1ECDC2EED2CCEEDFC2ECAE38F2C992411
:10160000AA24BB24682D8C2F0E949E09682D85E09A
:101610008C0F0E949E09FE2CED2CDC2CCC24CF5F7D
:10162000CE3361F76FEF83E40E949E096FEF84E48D
:101630000E949E096FEF85E40E949E096FEF86E489
:101640000E949E09DD2311F066E002C060918105D1
:101650008DE60E949E0960E089E70E949E096091E4
:1016600082058AE70E949E0960E083E70E949E0946
:1016700060E084E70E949E09D11109C0609179055C
:1016800070917A0580917B0590917C0504C060EC97
:1016900072E98DEE99E10E940D0ADF91CF91FF90E2
:1016A000EF90DF90CF90BF90AF909F908F90089574
:1016B00061E087E00E949E0964E28EE70E949E0935
:1016C00063E088E00E949E0960E088E00E949E0935
:1016D00065E087E00E949E0962E085E00E949E0925
:1016E00083E00E94980980936F0584E00E94980926
:1016F00080936E05089583E00E94980980936F059A
:1017000084E00E94980980936E0561E087E00E9462
:101710009E096AE070E080E090E00E94AF280E949D
:10172000580B00000895CF92DF92FF920F931F9302
:10173000CF93DF931F92CDB7DEB7082F162F8EE31E
:1017400099830E949E09F02EC02E9981D92E8C2D4E
:101750008F19811738F4F60161916F018FE70E94AC
:101760009E09F5CF64E085E00E949E0983E00E9417
:10177000980980936F0584E00E94980980936E0514
:101780000E948C2860936A0570936B0580936C05AA
:1017900090936D0569E087E00E949E0981E0809347
:1017A00071050F90DF91CF911F910F91FF90DF9006
:1017B000CF9008950F931F930E94930B8091710512
:1017C000813099F40E948C2800916A0510916B0574
:1017D00020916C0530916D05601B710B820B930B92
:1017E000603A76488140910548F3809171058130D7
:1017F00031F46DE971E080EE95E00E945B2A1F9163
:101800000F9108950F931F9380917105823021F4F9
:101810001092710581E020C0809171058130D9F46A
:101820000E948C2800916A0510916B0520916C052F
:1018300030916D05601B710B820B930B613A7648FA
:101840008140910540F061E087E00E949E0910927E
:10185000710582E001C080E01F910F910895CF9340
:10186000DF93EC014AE050E06D2F70E080EE95E0F0
:101870000E94292B6EE280EE95E00E942D2ABE0187
:1018800084E0769567958A95E1F76F7077274AE04F
:1018900050E080EE95E00E94292B6EE280EE95E00C
:1018A0000E942D2ABE016F7077274AE050E080EE3B
:1018B00095E00E94292BDF91CF910895D82FC0E0A9
:1018C000CD1780F42C9A64E670E080E090E00E94EE
:1018D000AF282C9864E670E080E090E00E94AF288A
:1018E000CF5FEECF6CE271E080E090E00E94AF2825
:1018F000E6CF0F931F93CF93DF93EC01062F15E0F4
:10190000115051F0CE010E942430081741F0602F91
:10191000CE010E942C30F4CF82E00E945E0CDF9159
:10192000CF911F910F910895A0E0B0E0EAE9FCE0AB
:101930000C940A2E482E562EC0E0D0E0612C712C5B
:10194000E12CF12C00E010E041100CC06090D205B9
:1019500086E4689E3001112459E1E52EF12C08EB54
:1019600015E01EC091E049120FC06090D205E6E478
:101970006E9E30011124FBE16F0E711C49E2E42ED2
:10198000F12C04E715E00CC082E0481209C028E100
:10199000622E77247394EE24E394F12C01ED15E08C
:1019A00043018C0E9D1E1092730510927205340136
:1019B000A62CA818B12CC30101966C01AE14BF046B
:1019C000A8F4A00EB11E511006C0C3010E9424301D
:1019D000F501808305C0F5016081C3010E94790C87
:1019E000F50180810E9461063601E2CFC3015110EA
:1019F00018C0C3010E942430B82EC6010E942430B2
:101A00002B2D30E0322F2227282B809172059091C8
:101A100073058217930779F4C0E0D0E055245394FE
:101A200093CF3601609173050E94790C6091720525
:101A3000C6010E94790CC05EDE4FC13E92E0D9071C
:101A400008F482CF852DCDB7DEB7E0E10C94262EC9
:101A500061E082E00E94940C089560E082E00E94C0
:101A6000940C8091D105853020F01092D1050E9410
:101A7000280D8091D1058093D205089561E080E022
:101A80000E94940C61E081E00E94940C089560E053
:101A900080E00E94940C882351F060E081E00E9475
:101AA000940C882321F080917405883349F00E94BA
:101AB000BF060E947A0681E00E94DF060E943E0D6A
:101AC0000895882319F069EA71E002C06DEA71E0B7
:101AD00080EE95E00E945B2A0895FF920F931F937A
:101AE000CF93DF9369EC7BE080EE95E00E94072ABC
:101AF0004091790550917A0560917B0570917C0544
:101B00002AE030E080EE95E00E94302B63EB7BE032
:101B100080EE95E00E94072A40917D0550917E0558
:101B200060917F057091800520E130E080EE95E0C6
:101B30000E94302B6DE97BE080EE95E00E94072A41
:101B40004AE050E06091810580EE95E00E94582BBC
:101B500067E87BE080EE95E00E94072A4AE050E0CB
:101B60006091820580EE95E00E94582B61E77BE052
:101B700080EE95E00E94072AC3E8D5E0F12C8E01A3
:101B800088818823A9F0FF2031F060EB71E080EEBE
:101B900095E00E942A2A21964AE050E0F8016081EF
:101BA00080EE95E00E94212BF394F8E1FF12E7CF3D
:101BB00080EE95E00E94352A6BE57BE080EE95E0B3
:101BC0000E94072A4AE050E060919B0580EE95E074
:101BD0000E94582B66E47BE080EE95E00E94072A85
:101BE000E0919C05E770F0E0EE0FFF1FEF57FC4F10
:101BF0006081718180EE95E00E945B2A61E37BE069
:101C000080EE95E00E94072A80919C0588718830BB
:101C100069F028F4811113C068E27BE00CC08031C8
:101C200041F0883161F46CE07BE005C06CE17BE061
:101C300002C066E17BE080EE95E00E94492A68EFF1
:101C40007AE080EE95E00E94072A40917505509158
:101C5000760560917705709178052AE030E080EE96
:101C600095E00E94302B6FED7AE080EE95E00E94C7
:101C7000072A8091BD0580710E94610D66EC7AE0B3
:101C800080EE95E00E94072A8091BD0580740E9435
:101C9000610D6DEA7AE080EE95E00E94072A80915E
:101CA000BD0580720E94610D60E97AE080EE95E0EA
:101CB0000E94072A84E795E00E94F407AB01BC016B
:101CC0002AE030E080EE95E00E94122B6BE87AE08B
:101CD00080EE95E00E94072A84E795E00E94F407D1
:101CE0009B01AC0160E472E48FE090E00E94C72D9C
:101CF000BA01A9012AE030E080EE95E00E94122BA3
:101D000068E87AE080EE95E00E94492ACDB7DEB718
:101D1000E5E00C94312E8F929F92AF92BF92CF92BA
:101D2000DF92EF92FF92811107C06FE77AE080EEB9
:101D300095E00E94492A2FC090E00E94740724E693
:101D400030E040E050E00E94C72DCA01B9012AE00E
:101D500030E040E050E00E94C72D49015A016B017C
:101D60007C012AE030E0B501A40180EE95E00E94FC
:101D7000122B6EE280EE95E00E942D2A2AE030E0E0
:101D8000B701A60180EE95E00E94122B63E780EE7A
:101D900095E00E946D2AFF90EF90DF90CF90BF906A
:101DA000AF909F908F9008951F93CF93DF9365E737
:101DB0007AE080EE95E00E94072A80919D058130AF
:101DC00041F46CE57AE080EE95E00E94492A10E04B
:101DD00050C0823019F465E47AE0F5CF843019F40C
:101DE00061E37AE0F0CF853091F766E27AE0EBCFFD
:101DF000C12FD0E0C930D1050CF441C068E3610FB8
:101E000080EE95E00E942D2A6EE17AE080EE95E06A
:101E10000E94072ABE016F5F7F4F4AE050E080EECC
:101E200095E00E94F12A63E17AE080EE95E00E945D
:101E3000072AC356DA4FE981E03218F566E07AE006
:101E400080EE95E00E94072A8981803130F06CE6AF
:101E500073E080EE95E00E942A2A69816F7070E03D
:101E60006F5F7F4F4AE050E080EE95E00E94FA2AD3
:101E70001F5F80914605181708F4BACF0FC061E3C1
:101E8000BECFEF70F0E0EE0FFF1FEF56FC4F60810A
:101E9000718180EE95E00E945B2AEACF6BEE79E0DB
:101EA00080EE95E00E94072A8091B5050E948B0E76
:101EB00060ED79E080EE95E00E94072A8091B605FA
:101EC0000E948B0E65EB79E080EE95E00E94072A78
:101ED0008091B7050E948B0E6AE979E080EE95E06B
:101EE0000E94072A4091AD055091AE056091AF0563
:101EF0007091B005411551056105710539F12AE070
:101F000030E080EE95E00E94302B67E679E080EECD
:101F100095E00E94072A8091B1050E949907AB01C4
:101F2000BC012AE030E080EE95E00E94302B63E4B3
:101F300079E080EE95E00E94072A4AE050E0609147
:101F4000B20580EE95E00E94582B06C06AE379E066
:101F500080EE95E00E94492A6DE179E080EE95E0FF
:101F60000E94072A6091B3057091B4054AE050E0E1
:101F700080EE95E00E94422B60E079E080EE95E0F3
:101F80000E94072A6091AC05603450F470E06F5FE6
:101F90007F4F4AE050E080EE95E00E94FA2A06C0AA
:101FA00067EF78E080EE95E00E94492A6AED78E0DC
:101FB00080EE95E00E94072A8091AB0580FF03C068
:101FC00062EB71E002C066EB71E080EE95E00E948A
:101FD0005B2A6DEB78E080EE95E00E94072A809105
:101FE000AB0582700E94610D6EE978E080EE95E0AD
:101FF0000E94072A8091AB0584700E94610D6FE7F3
:1020000078E080EE95E00E94072A8091AB05887009
:102010000E94610DDF91CF911F9108950F931F933F
:10202000CF93DF93209143052F3FA9F56FEF75E024
:1020300080EE95E00E94072A84E893E00E942F0C2E
:102040006EED75E080EE95E00E94072A80914405D0
:10205000909145050E942F0C6BEA75E080EE95E0AB
:102060000E94492A68E875E080EE95E00E94492ABE
:1020700060E775E080EE95E00E94492A6BE475E028
:1020800080EE95E00E94492A80EE95E00E94352A74
:102090000E94D40E68C012160CF065C0332727FDCD
:1020A00030958091460590E0821793070CF45BC051
:1020B00066E375E080EE95E00E94072A6091430593
:1020C000772767FD70954AE050E080EE95E00E942A
:1020D000FA2A6BE075E080EE95E00E94072A10E096
:1020E00008E2809147051817D0F5C12FD0E0CC0F3A
:1020F000DD1FC85BDA4F288130E0809143059927C6
:1021000087FD909501972817390739F56AEB71E03B
:1021100080EE95E00E942A2A4AE050E0602F80EE8F
:1021200095E00E94212B6EEB71E080EE95E00E941D
:102130002A2AE981EF70F0E0EE0FFF1FEF56FC4F07
:102140006081718180EE95E00E942A2A62EC71E044
:1021500080EE95E00E942A2A0F5F1F5FC2CF80EEBB
:1021600095E00E94352ADF91CF911F910F9108953C
:10217000FF920F931F93CF93DF93C3E8D5E0F12C29
:102180008E0188818823D1F164EC71E080EE95E0C6
:102190000E942A2A4AE050E06F2D80EE95E00E94CE
:1021A000212B61ED71E080EE95E00E942A2A2196B4
:1021B000F801208130E0A0E1B7E20E94812D9B016F
:1021C000AC01A0918205B0E00E94902DAB01BC0152
:1021D0008091790590917A05A0917B05B0917C055D
:1021E000480F591F6A1F7B1F2AE030E080EE95E000
:1021F0000E94302BF394F8E1FF12C2CFCDB7DEB7C7
:10220000E5E00C94312E1092DD0485E6EEEDF4E06D
:10221000DF011D928A95E9F70895CF93C82F8F3774
:1022200019F0883009F045C0E091DD04EE23D9F1C2
:10223000E150E093DD04F0E0E252FB4F10826DE0EC
:1022400070E080EE95E00E945906C0E08091DD04C8
:10225000C81760F4EC2FF0E0E252FB4F608170E0B1
:1022600080EE95E00E945906CF5FF0CF60E270E00B
:1022700080EE95E00E9459066DE070E080EE95E0FA
:102280000E945906C0E08091DD04C81778F5EC2F54
:10229000F0E0E252FB4F608170E080EE95E00E943A
:1022A0005906CF5FF0CF67E080EE95E00E942D2ABF
:1022B0001DC08B3119F40E9403111AC08D30C1F07A
:1022C0008A30B1F08091DD04843668F76C2F70E0BD
:1022D00080EE95E00E945906E091DD0481E08E0FCA
:1022E0008093DD04F0E0E252FB4FC08380E001C048
:1022F00081E0CF910895CF93C82F0E948C286093DE
:10230000C6047093C7048093C8049093C904C09313
:10231000DB04CC2329F040E051EE60E070E004C023
:1023200040E855E260E070E080EE95E00E94B72C56
:10233000CF9108959091CA04492F4F7050E0BA018F
:102340006F5F7F4F292F30E0E4E035952795EA95C0
:10235000E1F76217730759F0FA01E553FB4F8083E9
:1023600081E0890F8F70907F892B8093CA04089534
:102370006EE770E080EE95E00E9459060895A3E1B3
:10238000B1E0E5ECF1E10C940B2EE3E8F5E0712C03
:102390008191882321F0739428E17212F9CF65EDC1
:1023A00071E080EE95E00E945B2A4AE050E0672DE4
:1023B00080EE95E00E94582B80E00E947D0A0E94EA
:1023C000580B8E010E5F1F4FC12CD12C7601C39488
:1023D00066246A945C2C0E9480284B015C01209149
:1023E000820530E0A0E1B7E20E94812D9B01AC01A3
:1023F000C701B6010E94A32D2091790530917A057D
:1024000040917B0550917C05620F731F841F951FBF
:102410002091B9053091BA054091BB055091BC059A
:10242000261737074807590718F4F801608225C0B6
:102430008C2D0E94B10961E070E080E090E00E9484
:10244000AF28F80110820E948028681979098A094A
:102450009B09643F71408105910540F40E94C709C2
:10246000F8019081981778F78083EDCF50FE03C074
:102470002B982C9A02C02B9A2C982FEFC21AD20AB2
:10248000E20AF20A0F5F1F4F8FEFC816D104E10472
:10249000F10409F09FCFCE019395FC01D82E7FEF78
:1024A00068EC2E2F281B271510F051E056C0DE01D6
:1024B000129651E02FEF41E03D91321710F0322F8C
:1024C00001C0452F5F5F5F3F11F0232FF5CF419390
:1024D000242F30E0A1E0B0E0AC0FBD1FA20FB31F6E
:1024E0005C93413079F0DE01A20FB31F5C93423060
:1024F00049F0AFEFBFEFAC0FBD1FA20FB31F6C933E
:102500004E3F78F6A2E0B0E0AC0FBD1FA20FB31FA4
:102510007C934D3F30F6A3E0B0E0AC0FBD1FA20F9F
:10252000B31F6C93BECF452F242F30E0FC01E20F88
:10253000F31F6081AFEFB0E0AC0FBD1FA20FB31F60
:102540002C91621748F44150DC01A40FB11D2C916D
:1025500020836C934111E8CF5F5F571520F3372D2F
:10256000369520E0231770F4DC01A20FB11D4C91C9
:10257000522F530FFC01E50FF11D50815C934083F6
:102580002E5FF0CFF3E8EF2EF5E0FF2E8C01802FC9
:102590008D19871598F4F801C1908F014AE050E039
:1025A0006C2D80EE95E00E94212B6CE280EE95E090
:1025B0000E942D2AF701C1927F01E9CF80EE95E0BC
:1025C0000E94352A81E0CD5EDE4FEFE00C94272E8D
:1025D0001F920F920FB60F9211240F931F932F93F8
:1025E0003F934F935F936F937F938F939F93AF939B
:1025F000BF93EF93FF934091BD055091BE0560914D
:10260000BF057091C00586B18A019B010074112736
:102610002227332785FB882780F990E0A0E0B0E0EF
:10262000081719072A073B0709F468C0809184003E
:102630009091850010928500109284002091A7044B
:1026400021115CC045FD02C096958795853C29E027
:102650009207C0F180910A0190E0A0E0B0E00CE1A7
:1026600076956795579547950A95D1F74115510588
:102670006105710521F441E050E060E070E0481729
:1026800059076A077B07D8F480910A018F3FB9F098
:1026900040E080910A01481780F4842F90E0880F71
:1026A000991FFC01E957FB4F20813181FC01E55F57
:1026B000FE4F318320834F5FECCF1092A80410921D
:1026C0000A011CC08D3B22E09207A8F020910A016C
:1026D000203188F410910A0121E0210F20930A0192
:1026E0000E94DE08E12FF0E0EE0FFF1FE957FB4FDD
:1026F0009183808303C08FEF80930A01FF91EF9154
:10270000BF91AF919F918F917F916F915F914F9109
:102710003F912F911F910F910F900FBE0F901F901F
:10272000189583E0809380008AE1809381008FEF89
:102730009FEF909389008093880010926F0080E251
:1027400080936C00E8E6F0E08081826080830895E9
:102750000E942D0D8091D205843011F41092D20583
:1027600008956F3018F086958058089589E0689F25
:10277000802D11240895A0E0B0E0E1ECF3E10C9489
:10278000122EC82F0E948C28009138041091390411
:1027900020913A0430913B046B017C01C01AD10AAC
:1027A000E20AF30A9701860149E8C41643E1D40618
:1027B000E104F10410F010923C046093380470932B
:1027C000390480933A0490933B042091A7048FEF3F
:1027D000820F8230D8F5E0913C04EE2309F44EC11B
:1027E000E13011F482E0B8C1E03108F034C181E099
:1027F0008E0F80933C04F0E0E957FB4FC08380319B
:1028000009F0ACC1E9E8F4E0213029F4A181A695F2
:10281000A695808108C080819181A92FA695A69553
:10282000A69596958795A03148F4B0E090E0AA0F60
:10283000BB1FA55FBE4F11969C938E931092A80468
:10284000329684E0E739F807F9F688C1233009F0B9
:1028500005C1E0913C04E11104C0CF3009F07EC114
:102860000DC1E83148F481E08E0F80933C04F0E024
:10287000EA57FB4FC08372C1E83109F0ECC0C111C7
:10288000EAC040E050E0ABE0CA01B3E0880F991F16
:10289000BA95E1F7A49F9001A59F300D1124F9018D
:1028A000E957FB4F6081E1817E2F777075956795C1
:1028B000FC01EE0FFF1FE55FFE4F71836083F9019E
:1028C000E857FB4FB081B695B695B695E181FE2FDE
:1028D000F295FF0FF07E6F2F6B2BE695E695E69550
:1028E0007E2F777075956795FC01EE0FFF1FE35FF4
:1028F000FE4F71836083F901E757FB4FB081B295BA
:10290000B695B695B370C181DC2FDD0FDD0F6D2F4D
:102910006B2BC295C695C695C370E281E170EE0F30
:10292000EE0F7E2F7C2B75956795FC01EE0FFF1F38
:10293000E15FFE4F71836083F901E557FB4FB08182
:10294000B695E181FE2FF795FF27F7956F2F6B2B3B
:10295000E6957E2F777075956795FC01EE0FFF1F4A
:10296000EF5EFE4F71836083F901E457FB4FB08146
:10297000B295BF70E181FE2FF295F07F6F2F6B2B28
:10298000E295EF707E2F777075956795FC01EE0FDD
:10299000FF1FED5EFE4F71836083F901E357FB4F2C
:1029A000B081BB1FBB27BB1FC181DC2FDD0F6D2F8B
:1029B0006B2BCC1FCC27CC1FE281E370EE0F7E2F58
:1029C0007C2B75956795FC01EE0FFF1FEB5EFE4FAC
:1029D00071836083F901E157FB4FB081B695B695DD
:1029E000E181FE2FF295FF0FFF0FF07C6F2F6B2B15
:1029F000E695E6957E2F777075956795FC01EE0F4D
:102A0000FF1FE95EFE4F71836083F901E057FB4FC2
:102A100020812295269527703181E32FEE0FEE0F4E
:102A2000EE0F6E2F622B732F7295769577707595DA
:102A30006795FC01EE0FFF1FE75EFE4F7183608319
:102A40004F5F5F4F4230510509F01ECF80919D04CA
:102A500083FF1092A80410923C0480C0243009F037
:102A60007DC060913C0461110BC0C83AB1F4109272
:102A700073051092720588EA0E94610681E06CC0BD
:102A8000613019F4C093370404C0623031F4C0934C
:102A900036048C2F0E9461065AC0E09136042E2F16
:102AA00030E0220F331F462F50E0C90102968417F1
:102AB00095073CF0633268F7FA01EC57FB4FC0838F
:102AC000E8CF2D5F3F4F8C2F90E0609172057091A1
:102AD00073054217530749F4982F882786279727AD
:102AE000909373058093720532C06817790769F572
:102AF00080913704813049F5E13118F080E180930D
:102B00003604F0903604C8E8D4E000E010E00F1579
:102B1000D0F4FE013197808190E0982F882728819A
:102B2000822B43E0969587954A95E1F70E94DE084F
:102B3000F801EE0FFF1FE55FFE4F918380830F5F6B
:102B40001F4F2296E4CF1092A80410923C0480916B
:102B50003C04882319F08F5F80933C04CDB7DEB727
:102B6000E8E00C942E2EE82FF0E0E854FA4FE185CF
:102B7000E03150F4F894F0E0EE0FFF1FE55FFE4FF8
:102B800080819181789408958EE08E0F8B3058F477
:102B9000F0E0E25FF10924E62E9FC0012F9F900D27
:102BA00011240C960895E13F59F018F4E03F89F0A4
:102BB00004C0ED3F41F0EE3F49F080E092E008951F
:102BC00086E090E008958AEF93E008958FEF93E018
:102BD000089580E090E00895A2E2B0E0E2EFF5E130
:102BE0000C94082E9E012F5F3F4F80E1D9011D926A
:102BF0008A95E9F763E072E080EE95E029A33AA3B5
:102C00000E945B2A0E947B0B1D8A1E8A1F8A188ED7
:102C1000312C212C00E0812C912C540170E4472EA2
:102C200071EE572E7DE9672E78E1772EE0E5CE2E06
:102C3000E3ECDE2EE12CF12C84EF91E0A0E0B0E09B
:102C40008D8F9E8FAF8FB8A380EC91EDA8E9BBE18B
:102C5000898F9A8FAB8FBC8F80E491EEADE9B8E19C
:102C6000898B9A8BAB8BBC8B80EE95E00E946F2B8F
:102C7000892B09F4E1C080EE95E00E949C2B9C0119
:102C800033272C32310509F442C0ACF4233231052C
:102C900009F0ABC019821A821B821C821D821E821F
:102CA0001F82188619861A861B861C861D861E861C
:102CB0001F86188A60C02434310529F02335310578
:102CC00009F4B2C092C064E480EE95E00E942D2A1F
:102CD0002AE030E040E451EE6DE978E180EE95E0E5
:102CE0000E94BB2A6CE280EE95E00E942D2A2AE029
:102CF00030E040EC51ED68E97BE180EE95E00E9428
:102D0000BB2A6CE280EE95E00E946D2AADCF0F5F8A
:102D1000043009F0A9CF29813A814B815C81A8EE6A
:102D2000B3E00E94902D698B7A8B8B8B9C8B2D81CD
:102D30003E814F8158850E94902D698F7A8F8B8FAD
:102D40009C8F29853A854B855C852D8F3E8F4F8FD3
:102D500058A32D853E854F8558890E94902D6B0183
:102D60007C0160323EE473078105910530F462E333
:102D70008CE10E949E0900E077CF603345E774073D
:102D80008105910510F462E2F3CF60345CE97507C8
:102D90008105910510F466E2EBCF80E5C81683EC5F
:102DA000D806E104F10410F462E1E2CF90E6C9161E
:102DB0009AEED906E104F10410F465E1D9CFA0E759
:102DC000CA16A1E1DA06A1E0EA06F10410F461E016
:102DD000CFCFB0EACB16B6E8DB06B1E0EB06F104E4
:102DE00010F463E0C5CF65E0C3CF10ED180F1A30C3
:102DF00008F03ACFE1E0F0E0EC0FFD1F24E0029F85
:102E0000E00DF11D11242081318142815381AAE01E
:102E1000B0E00E94902D610F711D811D911D608396
:102E200071838283938320CF49885A886B887C88FA
:102E3000812C912C540118CF81149104A104B10468
:102E400089F4C301B2010E940D0A61E070E080E0E4
:102E500090E00E94AF281D8A1E8A1F8A188E312C8E
:102E600022242A948D8D9E8DAF8DB8A18816990647
:102E7000AA06BB06D0F40E94C7092D893E894F8956
:102E8000588D280F311D411D511D2D8B3E8B4F8BB1
:102E9000588F381608F4382E821508F4282E3FEF84
:102EA000831A930AA30AB30A56C0C301B20128EEDB
:102EB00033E040E050E00E94C72DBA01A9012AE0AA
:102EC00030E080EE95E00E94122B6CE280EE95E0FF
:102ED0000E942D2A4AE050E0632D80EE95E00E948A
:102EE000212B6CE280EE95E00E942D2A6D897E896F
:102EF0008F89988DA50194010E94C72DBA01A9015F
:102F00002AE030E080EE95E00E94122B6CE280EE29
:102F100095E00E942D2A4AE050E0622D80EE95E077
:102F20000E94212B6CE280EE95E00E946D2A4C0CF1
:102F30005D1C6E1C7F1C898D9A8DAB8DBC8D84159C
:102F40009505A605B70520F449885A886B887C88C2
:102F5000812C912C540129893A894B895C89283E1E
:102F600033404105510509F07FCEA296E2E10C9471
:102F7000242EACE1B0E0EFEBF7E10C94122E0E94AE
:102F80008C286B017C0181E00E947D0A14E703E03C
:102F9000198361E0CE0101960E94DA0B009371055E
:102FA0000E94580B6AEF70E080E090E00E94AF282A
:102FB00080917105833089F480EE95E00E946F2B3B
:102FC000892B59F40E948C286C197D098E099F0960
:102FD0006038734C894C9140D8F2809171058330F0
:102FE00009F44FC08FE70E9476090E9489098983FE
:102FF000843511F083E05CC00E9489091092440579
:10300000809345050E94890920914405309145052A
:10301000280F311D30934505209344050E948909EE
:10302000809346050E94890980934705813110F7F6
:10303000F12C0F2D10E08091470590E0880F991F2B
:103040000817190740F40E948909F801E85BFA4F54
:103050008083F394EECF80E7898361E0CE0101960F
:103060000E94DA0B83E0809371050E94580B62E3A3
:1030700070E080E090E00E94AF288091710583307D
:1030800011F482E015C08FE70E9476090E94890939
:103090008983803509F0AECF0DE915E00E948909DA
:1030A000F80181938F01F5E0083B1F07B9F781E034
:1030B0006C96E8E00C942E2E80914305992787FDAD
:1030C0009095A92FB92FFC013196EB30F10508F04E
:1030D00066C0EC5CFF4F0C943F2E62E778E080EE18
:1030E00095E00E94492A84E893E00E942F0C6AE54B
:1030F00078E080EE95E00E94492A65E378E080EE72
:1031000095E00E94492A6BE078E080EE95E00E940D
:10311000492A6AEE77E080EE95E00E94492A6DEB3D
:1031200077E080EE95E00E94492A67E977E080EE3B
:1031300095E00E94492A63E777E080EE95E00E94DF
:10314000492A6CE477E080EE95E00E94492A80EEFF
:1031500095E00E94352A0E946D0D21C06FE277E054
:103160001AC06AE077E017C065EF76E014C066ED3C
:1031700076E011C062E976E00EC06DE776E00BC044
:1031800068E676E080EE95E00E94492A62E276E009
:1031900002C06CE076E080EE95E00E94492A6AE089
:1031A00070E080E090E00E94AF2880EE95E00E9401
:1031B0006F2B892B29F080EE95E00E949C2BF5CF98
:1031C0000895ACE1B0E0E7EEF8E10C94122E909196
:1031D00043059F3F09F023C1482F50E0FA013A9779
:1031E000EF36F10508F00FC1E15CFF4F0C943F2E64
:1031F00060E172E0A0C06CE172E080EE95E00E94B8
:103200005B2A85E789838BE1EDE9F5E0DE01129623
:1032100001900D928A95E1F76CE1CE0101960E9432
:10322000DA0B0E94580B83E08093710568EC70E024
:1032300080E090E00E94AF2880917105843009F011
:10324000E2C08FE70E9476090E948909898385354B
:1032500009F0D9C06DEE74E080EE95E00E94492A35
:103260006FEC74E080EE95E00E94492A61EB74E017
:1032700096C064E372E080EE95E00E945B2A89E6E6
:10328000898361E0CE0101960E94DA0B0E94580BFF
:1032900083E08093710568EC70E080E090E00E942C
:1032A000AF2880917105843009F0ADC08FE70E948E
:1032B00076090E94890989838E010E5F1F4F7E0166
:1032C0004DE1E40EF11C0E948909F80181938F0100
:1032D000EE15FF05C1F78BE1FE013296ADE9B5E0D1
:1032E00001900D928A95E1F78981893409F08BC0AC
:1032F00063E974E080EE95E00E94492A65E774E096
:1033000080EE95E00E94492A67E574E048C06EE4CB
:1033100072E080EE95E00E945B2A8EEF8093430579
:1033200072C080528750805390914605981708F0DC
:1033300066C06DE572E080EE95E00E945B2A63C096
:1033400084E18093430560E274E029C085E18093C5
:10335000430569EE73E023C086E18093430562EB89
:1033600073E01DC087E18093430568E673E017C0F2
:1033700088E18093430567E573E011C089E180939C
:10338000430563E473E00BC08AE1809343056EE27A
:1033900073E005C08BE18093430566E073E080EE47
:1033A00095E00E94492A2FC06CEE72E080EE95E015
:1033B0000E94492A8091AB0591E01DC066ED72E044
:1033C00080EE95E00E94492A8091AB0592E013C0FF
:1033D00061EC72E080EE95E00E94492A8091AB0595
:1033E00094E009C066EA72E080EE95E00E94492A06
:1033F0008091AB0598E089278093AB058FEF809390
:1034000043050E940E1080EE95E00E946F2B892BE1
:1034100009F45BC180EE95E00E949C2BF4CF0E94E2
:103420000D11882309F451C18091DD04811104C07C
:103430008FEF8093430541C140E050E060E070E0D1
:103440008EED94E00E94B62E40914305042F112783
:1034500007FD1095212F312FF8013197EB31F10540
:1034600008F01BC1E255FF4F0C943F2E552747FD36
:1034700050952091460530E0241735070CF40DC116
:103480008B019C01015011092109310900321105FC
:103490002105310558F0C0904705E9E4F5E0F12C2D
:1034A000D12CA8E2EA2E415051090FC0FA01E3568F
:1034B000FA4F61506083D9C0DF0111972C9130E041
:1034C0002417350729F0F3943296FC10F5CFCBC0C2
:1034D0000E2D10E020E030E0061717072807390707
:1034E00041F42081DA01A356BA4F11962C93DD24C2
:1034F000D394E394E8CF6F3F71058105910511F0F6
:1035000008F0CBC06093B505B0C06F3F7105810571
:10351000910511F008F0C1C06093B605A6C06F3FD9
:1035200071058105910511F008F0B7C06093B705EA
:103530009CC02091DE0420622037E9F440E050E096
:1035400060E070E08FED94E00E94B62E9B01AC012C
:10355000DC01CB010197A109B1090897A105B105CB
:1035600008F0AEC0A4EDB0E30E94902D6A5E7C4AE4
:103570008A46954E24C02636E9F440E050E060E0EB
:1035800070E08FED94E00E94B62E9B01AC01DC014F
:10359000CB010197A109B1090797A105B10508F071
:1035A0008FC0A8EAB1E60E94902D645E7C438E46EF
:1035B000944E05C0611571058105910579F08B0167
:1035C0009C010054114E2D4938410138F0EF1F077E
:1035D000FAEF2F07F2E03F0708F05FC06093AD05F8
:1035E0007093AE058093AF059093B0053EC06F3FDA
:1035F00071058105910511F008F04FC06093B10588
:1036000034C08B019C0101501109210931090F3F80
:1036100011052105310508F040C06093B20525C0B1
:103620008B019C01045C1940210931090D344DE1E5
:1036300014072105310528F47093B4056093B30590
:1036400014C0611571058105910521F48FEF8093F8
:10365000AC050BC06134710581059105F0F4615032
:103660006093AC0502C0DD20C1F08091DC048111C3
:103670001AC080917D0590917E05A0917F05B09143
:1036800080050196A11DB11D80937D0590937E0557
:10369000A0937F05B093800506C06FE672E080EED0
:1036A00095E00E945B2A0E9403118FEF80934305EF
:1036B0006AE080EE95E00E946D2A0E940E1005C01F
:1036C00061E070E080E090E07ACF6C96E8E00C94E6
:1036D0002E2E6AE572E080EE95E00E94492A62E4AF
:1036E00072E080EE95E00E94492A80EE95E00E940B
:1036F0006F2B892B31F080EE95E00E949C2B0E946D
:10370000E1180E94B917823029F0833051F46DE03E
:1037100072E002C064E272E080EE95E00E94492A05
:1037200008958FEF809343051092DC040E940E10E1
:10373000809143058E3F69F080EE95E00E946F2BEB
:10374000892BB1F380EE95E00E949C2B0E94E1183A
:10375000EFCF08950F931F93109143051F3F09F07A
:10376000D2C0893409F457C000F5883309F469C020
:1037700058F4803309F477C008F061C08B3109F444
:1037800040C08132B1F1B9C0813409F487C030F44E
:10379000893309F466C0803461F1AFC0823409F422
:1037A0008EC0863409F448C0A8C0823609F487C0A8
:1037B00078F4883531F128F48235C1F18335E1F0B0
:1037C0009CC08A3509F494C0813609F467C095C05D
:1037D000823761F128F4863679F18936E1F08DC0BF
:1037E000883779F08A3709F483C0833709F085C0B8
:1037F00003C060E172E015C00E943E0D6DE872E00A
:1038000004C00E94470D67EA72E080EE95E00E94D6
:103810005B2A8EEF70C00E947A060E94BF0666EC9B
:1038200072E080EE95E00E945B2A67C081E00E9412
:10383000DF066FED72E0F5CF0E94B8105EC08053D6
:103840005AC06AEF71E080EE95E00E94492A90919B
:103850009C0588E0890F8871977E892B80939C0551
:103860001AC089E048C067EE71E080EE95E00E94E2
:10387000492A8091BD059091BE05A091BF05B091E8
:10388000C00520E182278093BD059093BE05A093DB
:10389000BF05B093C005109343052FC061ED71E0E3
:1038A00080EE95E00E94492A8091BD059091BE0569
:1038B000A091BF05B091C00540E4842710C060EC22
:1038C00071E080EE95E00E94492A8091BD059091BB
:1038D000BE05A091BF05B091C00520E2822780936C
:1038E000BD059093BE05A093BF05B093C00502C06F
:1038F0000E94691B8FEF80934305809143058E3FA3
:1039000009F0D4C0DDC00E940D11882309F4D8C08D
:103910008091DD04811104C08FEF80934305C6C000
:1039200040E050E060E070E08EED94E00E94B62E42
:1039300000914305112707FD1095212F312FF80124
:103940003197E930F10508F0B4C0E753FF4F0C940C
:103950003F2E8B019C010154114E2D4938410F37E8
:10396000104F2A4F324008F0A4C06093790570933D
:103970007A0580937B0590937C0577C060937D05E5
:1039800070937E0580937F059093800581E08093FE
:10399000DC046BC0683071058105910508F089C0B1
:1039A0006093810562C08B019C01015011092109BE
:1039B00031090A3011052105310508F07AC06093FC
:1039C000820553C060EB71E08EED94E00E94F02F11
:1039D00010E0009799F00E94CA2F009779F01831F3
:1039E00030F4E12FF0E0EC58FA4F87871F5F60EB6F
:1039F00071E080E090E00E94F02FEBCF1831A8F545
:103A0000E12FF0E0EC58FA4F17861F5FF7CF6530D3
:103A100071058105910508F04CC060939B0525C098
:103A20008B019C0101501109210931090630110552
:103A300021053105F0F520919C05287F262B209348
:103A40009C0513C08B019C0101501109210931090A
:103A50000115124C2140310560F560937505709396
:103A6000760580937705909378058091DC04811129
:103A700013C080917D0590917E05A0917F05B09146
:103A800080050196A11DB11D80937D0590937E0553
:103A9000A0937F05B09380050E9403118FEF809360
:103AA00043056AE080EE95E00E946D2A0E945C1852
:103AB00007C06FE672E080EE95E00E945B2AECCFD3
:103AC0001F910F9108958FEF809343051092DC04AE
:103AD0000E945C18809143058E3F69F080EE95E06E
:103AE0000E946F2B892BB1F380EE95E00E949C2BF6
:103AF0000E94AA1BEFCF6AE070E080E090E00E9495
:103B0000AF2880EE95E00E946F2B892B29F080EE84
:103B100095E00E949C2BF5CF0895CF93C82F682F76
:103B200080EE95E00E94C92B909168059C279093A8
:103B30006805CF910895A1E0B0E0E1EAFDE10C94C1
:103B4000182E99830E948D1D9981892F0E948D1DA9
:103B50002196E2E00C94342E1F93CF93DF93182F1D
:103B6000EB011092680565EB70E080EE95E00E9435
:103B7000590662E670E080EE95E00E945906812FBA
:103B80000E948D1DCE010E949B1DDF91CF911F9140
:103B900008956091680580EE95E00E94C92B089514
:103BA000A1E2B0E0E6EDFDE10C94142E7B018A0168
:103BB0008C3009F452C108F040C0863009F4BCC012
:103BC00018F5833009F491C070F4813009F472C0A3
:103BD000823009F047C26BE170E082E00E94AC1DC8
:103BE0000DE915E078C0843009F487C0853009F00C
:103BF00039C26091470570E0660F771F85E00E942B
:103C0000AC1D08E415E086C0893009F4A7C070F443
:103C1000873009F49BC0883009F024C261E070E06D
:103C200088E00E94AC1D8091D20522C28A3009F43E
:103C3000CAC08B3009F4F1C015C28A3609F474C1C8
:103C4000D8F4873609F439C138F4853609F40DC142
:103C5000863609F41EC106C2883609F436C1893693
:103C600009F000C261E070E089E60E94AC1D0E948C
:103C70007A060E94BF06F4C18D3609F4D3C138F428
:103C80008B3609F490C18C3609F499C1EBC18E369C
:103C900009F4DBC1873C09F0E5C161E070E087EC25
:103CA0000E94AC1D81E00E948D1D0E94C91D1092D2
:103CB0006905E2C169E270E081E00E94AC1D04E7A1
:103CC00015E0F80181918F010E948D1DF5E00D39FD
:103CD0001F07B9F7CFC1F80181918F010E948D1D97
:103CE000F5E0083B1F07B9F7C5C161E070E083E06C
:103CF0000E94AC1D0E94B917BBC161E070E084E076
:103D00000E94AC1D81E00E948D1D0E94C91D0E9471
:103D1000EC15B2C18091470590E0880F991F98017A
:103D2000285435402817390708F0A4C1F8018191BB
:103D30008F010E948D1DEECF62E070E086E00E9450
:103D4000AC1D84E893E00E949B1D94C161E070E08B
:103D500087E00E94AC1D809146058AC186E6898372
:103D600061E0CE0101960E94DA0B0E94580B83E0BD
:103D70008093710568EC70E080E090E00E94AF28CD
:103D8000809171058430D9F48FE70E9476090E94F2
:103D900089098983863469F460E270E089E00E94D1
:103DA000AC1D10E20E9489090E948D1D1150D1F7AF
:103DB00061C161E070E089E00E94AC1D51C161E029
:103DC00070E089E052C169E170E08AE00E94AC1DB8
:103DD0001092B805209170058091BD059091BE05A7
:103DE000A091BF05B091C005222311F0806801C0E9
:103DF0008F778093BD059093BE05A093BF05B093C8
:103E0000C00508EB15E0F80181918F010E948D1D1E
:103E1000F5E0013D1F07B9F72DC161E270E08BE0CD
:103E20000E94AC1D8091A8048F3F39F08091A804B6
:103E300091E0980F9093A80402C08091A8040E947A
:103E40008D1D10E0812F0E94B3150E9409090E9468
:103E50009B1D1F5F1031B1F70DC161E070E08CE078
:103E60000E94AC1D8091D10503C161E070E085E640
:103E70000E94AC1D89E2E816F10409F0F8C0D801EF
:103E8000E4E7F5E08D91819385E0ED39F807D1F70E
:103E9000E7C061E070E086E60E94AC1DEBE1EE1643
:103EA000F10409F0E4C0D801EDE9F5E08D918193CA
:103EB00085E0E83BF807D1F7D3C061E070E087E622
:103EC0000E94AC1D0E943E0DCBC061E070E088E610
:103ED0000E94AC1D85E789838BE1EDE9F5E0DE0109
:103EE000129601900D928A95E1F76CE1CE01019650
:103EF0000E94DA0B0E94580B83E08093710560E208
:103F000073E080E090E00E94AF28809171058430DA
:103F100009F0ADC08FE70E9476090E948909898364
:103F2000853509F0A4C09CC061E070E08AE60E947B
:103F3000AC1D89E6898361E0CE0101960E94DA0B0F
:103F40000E94580B83E08093710560E273E080E08B
:103F500090E00E94AF2880917105843009F087C0FD
:103F60008FE70E9476090E94890989838E010E5F7E
:103F70001F4F7E01EDE1EE0EF11C0E948909F80150
:103F800081938F01EE15FF05C1F78BE1FE0132969B
:103F9000ADE9B5E001900D928A95E1F78981893408
:103FA00009F065C05DC061E070E08BE60E94AC1D69
:103FB000F80180818093D2050E94470D51C061E0D5
:103FC00070E08CE60E94AC1DF0E2EF16F10461F4A3
:103FD00087E6898380E2F801DE01129601900D9256
:103FE0008A95E1F761E203C087E4898361E0CE014D
:103FF00001960E94DA0B0E94580B83E080937105B2
:104000006CE474E080E090E00E94AF28809171053C
:10401000843069F58FE70E9476090E948909873408
:1040200031F51EC061E070E08DE60E94AC1D89E1B3
:10403000E816F104E1F4D801E8EBF5E08D91819305
:1040400085E0E13DF807D1F70BC061E070E08EE656
:104050000E94AC1DF80180818093D1050E94280D3B
:1040600081E006C061E070E08AEC0E94AC1D80E057
:104070000E948D1D0E94C91DA196E6E00C94302E71
:10408000A0E0B0E0E6E4F0E20C94122ECAECD3E03B
:1040900014E606E035E0F32E44E0E42E53E0D52E9E
:1040A00062E0C62E80EE95E00E946F2B892B09F40A
:1040B0009BC080EE95E00E949C2B282F80933504B6
:1040C0004091340450E04730510560F7FA01EE5258
:1040D000FF4F0C943F2E853B29F781E080933404F9
:1040E000E1CF823609F07DC0C0923404DBCF8093EB
:1040F000330480933204D0923404D4CF9C0133270C
:104100003093310420933004909132049827909397
:104110003204E0923404C6CF382F22274091300475
:1041200050913104242B352B3093310420933004EB
:1041300090913204982790933204F09234042536FB
:10414000310508F4AFCF61E070E08CEC0E94AC1D4B
:1041500081E00E948D1D0E94C91D43C020912E0444
:1041600030912F04F901E653FC4F80839091320483
:10417000982790933204C901019690932F0480935D
:104180002E0420913004309131048217930708F4F3
:1041900089CF0093340486CF8091320482130BC000
:1041A00060912E0470912F044AEC53E08091330407
:1041B0000E94D01D0DC062E070E08BEC0E94AC1D2F
:1041C000809133040E948D1D809168050E948D1D91
:1041D000FE01812F11928A95E9F710922F04109217
:1041E0002E04109234045ECFCDB7DEB7E8E00C9415
:1041F0002E2E81E08093690580916905882349F01E
:1042000080EE95E00E946F2B892BB1F30E94402035
:10421000F3CF0895AAE2B0E0E0E1F1E20C94102EB1
:104220000E9480286B017C0181E00E947D0A80EE63
:1042300095E00E946F2B892B29F080EE95E00E947B
:104240009C2BF5CF2C9811E072E6B72EE9E2AE2E4A
:1042500003E00E9480286C197D098E099F09693C42
:10426000710581059105D0F11123C1F10E948028CB
:104270006B017C012B9A80ED97E00E94A807B98220
:10428000E4E7F5E0DE0112968A2D01900D928A9501
:10429000E1F76AE2CE0101960E94DA0B2B9880E0EA
:1042A00090E00E94A807009371050E94580B62E3FA
:1042B00070E080E090E00E94AF288091710584302A
:1042C00061F4009371058FE70E9476090E948909C5
:1042D00011E0823419F410E001C011E08AE00E947C
:1042E000A529892B81F411E00EC02C9A2B9A80EE1F
:1042F00095E00E949C2B8D309105A9F05CF40A9703
:1043000091F02C982B9880EE95E00E946F2B892BD2
:1043100061F79FCF8332910579F08234910589F757
:104320000E94F920EECF62EB71E080EE95E00E94F2
:10433000492A0E94631DE5CF0E94EC15E2CF8F92BF
:104340009F92AF92BF92CF92DF92EF92FF921F9314
:10435000CF93DF938AE00E94A529892B09F089C0B9
:1043600068EC70E080E090E00E94AF2880E090E090
:104370000E94A8070E9480284B015C016B017C0110
:1043800080ECC80E82E1D81EE11CF11C0E9480283E
:104390006C157D058E059F0530F48AE00E94A529E5
:1043A000892BA1F364C08AE00E94A529892B09F01A
:1043B0005EC080ED97E00E94A8070E9480286B01F4
:1043C0007C01D0E0C1E088E4880E86E2981EA11C42
:1043D000B11C11E08AE00E94A529892B21F58C14DB
:1043E0009D04AE04BF0430F480ED97E00E94A8075E
:1043F000D1E0F0CF0E9480286C197D098E099F09B9
:10440000693C71058105910528F30E9480286B01A4
:104410007C01C12719F080ED97E002C080E090E0B8
:104420000E94A807D7CF80E090E00E94A807DD2374
:10443000B9F08091D10590E0019665E070E00E94AE
:10444000B32D8093D1050E94280D0E94A8130E94CD
:10445000470D64EF71E080E090E00E94AF2809C052
:1044600080E00E94DF060E94BF110E943E0D0E9464
:104470000A21DF91CF911F91FF90EF90DF90CF90B5
:10448000BF90AF909F908F900895CF92DF92EF9260
:10449000FF9280E00E94DA070E94B10761E08CE0A1
:1044A0000E94392961E08BE00E94392960E08AE0AE
:1044B0000E94392960E083E10E94392961E083E1AB
:1044C0000E94722961E082E10E94392960E082E164
:1044D0000E9472290E949F0740E052EC61E070E068
:1044E00080EE95E00E94B72C0E94A8130E94470D11
:1044F0000E9491138FEF8093A8040E94C6077894BE
:104500000E9480286B017C018091A8048F3F59F4A0
:104510000E9480286C197D098E099F09603D7740B3
:104520008105910588F380ED97E00E94A80761E07E
:104530008AE00E9472292C9A80EE95E00E946F2BEF
:10454000892B29F080EE95E00E949C2BF5CF6CEF33
:1045500072E080EE95E00E942A2A84E893E00E94AF
:104560002F0C63E173E080EE95E00E942A2A4AE076
:1045700050E060E070E080EE95E00E94FA2A62E38D
:1045800070E080E090E00E94AF2880EE95E00E940D
:104590006F2B04970CF180EE95E00E949C2B8234E7
:1045A0009105D1F480EE95E00E949C2B8E3491050C
:1045B00099F480EE95E00E949C2B8434910561F47F
:1045C00080EE95E00E949C2B819731F480E090E092
:1045D0000E94A8070E940A21409175055091760516
:1045E0006091770570917805DB01CA010197A109F7
:1045F000B1090497A105B10568F44093A7044330BD
:1046000029F440EA56E861E070E004C040E052EC72
:1046100061E070E080EE95E00E94B72C0E949F213F
:104620002C9880E090E00E94A8070E9491131092BD
:10463000C3048091BD0583FF11C080918905882343
:1046400051F080919005882331F08091970588235F
:1046500011F087E001C085E08093C30480E00E94F0
:104660007D0A8091C4040E94B1090E94580B1092E7
:104670003F0410923E0410923D04F12C8091D2052B
:104680008F15B0F062E370E080E090E00E94AF2808
:1046900080ED97E00E94A80762E370E080E090E080
:1046A0000E94AF2880E090E00E94A807F394E6CF34
:1046B00080919C0584FF08C0982F987181E0983103
:1046C00009F080E00E947B118FE00E94DA07FF90E2
:1046D000EF90DF90CF900895EF92FF920F931F938A
:1046E000CF93DF938C016EE770E080EE95E00E943F
:1046F0005906E801F12CF0E2EF2E8E0188818D57EA
:10470000823048F46DE770E080EE95E00E94590633
:1047100088818E2588832196F801608180EE95E05E
:104720000E94C92BF394F9E0FF12E7CF6EE770E027
:1047300080EE95E00E945906CDB7DEB7E6E00C9416
:10474000302EA9E0B0E0E7EAF3E20C94182E909145
:10475000C50491110EC09EEF99838A836B8350E04C
:10476000559547954C832D83198618861F821E8286
:104770002EC04091CA04842F90E0B4E095958795AF
:10478000BA95E1F7242F2F7030E08217930719F1C3
:104790008DEF89831B82FE01349650E0842F90E0D8
:1047A000A4E095958795AA95E1F7242F2F7030E026
:1047B0008217930749F0DC01A553BB4F8C9181937D
:1047C000405F5F5F563051F74093CA045A83CE0171
:1047D00001960E946C238091C50490E0019666E0EA
:1047E00070E00E94B32D8093C5042996E2E00C94FA
:1047F000342EA0E0B0E0EFEFF3E20C94112E6C0148
:104800006EE770E080EE95E00E9459068601E12C8B
:10481000F12CC0E0D0E030E2B32EF801608183E8F3
:10482000860F823078F46DE770E080EE95E00E94AC
:104830005906F80160816B2570E080EE95E00E94DA
:10484000590604C080EE95E00E94C92BE114F104E2
:1048500059F0F80180819E01280F311DC901C92F2F
:10486000DD27C80FD91FDD273FEFE31AF30A89E0E0
:10487000E816F10459F028E0E216F10421F48C2F37
:104880008095F60180870F5F1F4FC7CFCDB7DEB78A
:10489000E9E00C942D2EA9E0B0E0E1E5F4E20C94FF
:1048A000182EE82F362F8091C50490E0019664E21F
:1048B00070E00E94B32D8093C50458E9598350E1FC
:1048C0005A83813089F048F08230B9F08330D9F4CE
:1048D0008B8381EF8C833D8319C085E08B8381EFCF
:1048E0008C832F5F2D8312C08B8381EF8C8384E6B2
:1048F000489FA00111245D8309C084E08B8381EF70
:104900008C83ED8303C00E94B81104C0CE010196D0
:104910000E94F9232996E2E00C94342EA2E0B0E044
:10492000E4E9F4E20C940D2E182F762E2A834983A5
:104930000E948C286B017C018091DB048090C6046E
:104940009090C704A090C804B090C9042A814981FE
:104950008823C1F0D701C60188199909AA09BB09A2
:104960004C015D0191EE89169EE29906A104B10405
:1049700020F1241708F4422F202F672D812F0E9449
:104980004B2413C0D701C60188199909AA09BB098C
:104990004C015D0191E3891695E79906A104B104E4
:1049A00060F0672D812F0E94A123C092C604D0928F
:1049B000C704E092C804F092C9042296EDE00C947A
:1049C000292EA2E2B0E0E7EEF4E20C940E2E8CE089
:1049D0000E94980981110DC06BE173E080EE95E0B3
:1049E0000E945B2A2C9A80E00E947D0A0E94580B4C
:1049F0002C9880EE95E00E946F2B892B01F180EEC0
:104A000095E00E949C2B9091A704992319F00E9495
:104A1000BB13EFCF40913E0450E09A012F5F3F4F10
:104A20002F71332760913F0470E02617370709F391
:104A3000FA01E75BFB4F808320933E04DACF80913D
:104A40007105843009F086C00E948C2861157105BB
:104A50008105910549F06093B5047093B604809385
:104A6000B7049093B8040CC081E090E0A0E0B0E0FF
:104A70008093B5049093B604A093B704B093B804A0
:104A80008091AB049091AC0481609093AC048093CE
:104A9000AB0483E0809371058FE70E94760909E6F5
:104AA00014E00E948909F80181938F01F4E0023734
:104AB0001F07B9F72091720480916904982F9227FB
:104AC00096FF3BC090E4922790937204982F9873BE
:104AD0009833F1F410E0212F30E080916904877061
:104AE00090E0821793074CF11F5F20919C05812F66
:104AF00090E0FC01E759FB4F24FF04C080810E9435
:104B00009A11E9CF608180EE95E00E94C92BE3CF36
:104B10008F7399F480916A048093B40480916B043C
:104B20008093B20480916C048093B10480916F04EF
:104B300090E09093AA048093A90480913D04813071
:104B400019F482E080933D0480913D04833011F498
:104B500010923D040E948C286B017C018091AD0471
:104B60009091AE04A091AF04B091B0040097A1055C
:104B7000B105C9F0A7019601281B390B4A0B5B0B45
:104B8000DA01C901883B9B40A105B10560F00E9494
:104B9000C7098093B3041092AD041092AE04109232
:104BA000AF041092B0048091B9049091BA04A0911E
:104BB000BB04B091BC0446015701881A990AAA0A9D
:104BC000BB0A84E795E00E94F40786169706A806BC
:104BD000B90608F4A8C0C092B904D092BA04E09211
:104BE000BB04F092BC040E9457068091A804883050
:104BF000A0F08091BD059091BE05A091BF05B09138
:104C0000C0055CE1B695A795979587955A95D1F71C
:104C1000892B8A2B8B2B09F09EC18091A8048F5F72
:104C20008093A8048091B5049091B604A091B70434
:104C3000B091B8040097A105B105F1F0C81AD90ADE
:104C4000EA0AFB0A84E795E00E94F4076C157D05EB
:104C50008E059F0508F006C18091BD0584FD04C046
:104C600080ED97E00E94A8071092B5041092B60458
:104C70001092B7041092B80490917204907C9093B3
:104C8000720450913E0480913F0420913D045817D6
:104C900009F405C1223009F002C1905890937204C2
:104CA000E0919C05E770F0E0E758FC4F60816930C7
:104CB00008F0DDC0615040E04613DBC080933F0444
:104CC00087E3840F90917204892B80937204409340
:104CD000400483E080933D042B9A8091810590915C
:104CE000C304911129C10E94780A8091C4040E94D2
:104CF000B109E0919C05E770F0E0E758FC4F608156
:104D000082E794E00E94930BE091C404EF5FE0938C
:104D1000C404E83109F41CC1F0E0EC58FA4F87856F
:104D2000882309F415C10E94020C813069F5809135
:104D30009C05887149F18091AB049091AC04880F77
:104D4000991F9093AC048093AB0483E0809371052A
:104D50000E94580B0E948C286093AD047093AE049F
:104D60008093AF049093B004672B682B692B61F498
:104D700081E090E0A0E0B0E08093AD049093AE04B9
:104D8000A093AF04B093B00480919C0584FF1FC032
:104D90008091AB049091AC048E7F0E942A09182F59
:104DA0006091A9048091B4040E94B113482F612F2F
:104DB0008091B30449A30E94B1130091D205282F1A
:104DC00049A16091B1048091B2040E948E242B9875
:104DD0008091C1048130C1F018F08230B1F1C8C0B7
:104DE0008AE00E94A529892B09F0C2C081E0809346
:104DF000C1040E9480286093BD047093BE04809318
:104E0000BF049093C004B4C08AE00E94A529892BF6
:104E100031F50E948028C090BD04D090BE04E0907F
:104E2000BF04F090C0046C197D098E099F09693E8A
:104E300073408105910508F49BC082E08093C10412
:104E400080ED97E00E94A80793C08AE00E94A52900
:104E5000892B09F48DC080E090E00E94A807109291
:104E6000C10486C080E090E00E94A80705CF68E0FA
:104E700022CF851709F422CF4F5F242F30E090E036
:104E8000F901EE58FB4FDC01A75BBB4F7C917083AF
:104E9000F901E05CFB4F708301968F710DCF2430D8
:104EA000B1F42091400481E494E0A3E7B4E0FC0174
:104EB0003E2F381B321718F431913D93F9CF87E319
:104EC000820F90917204892B8093720402CF80919B
:104ED000C104823051F49160909372042C9A8E0137
:104EE0000F5F1F4FF12CB80110C02C9880913D042A
:104EF000811103C081E080933D0480913D048330A3
:104F000071F784E080933D04EACF8F2D69A37AA3E3
:104F10000E94B315F801819391938F01F39469A1D5
:104F20007AA1F0E1FF12F1CF80919C0543E754E0B4
:104F300087700E947908D0CE882309F4D4CE2091BE
:104F4000C20431E0320F3093C2042913CCCE0CC01E
:104F50001092C404E8CE8091A804883009F42C9AF9
:104F600089E08093A804DFCE1092C2048150BBCEAA
:104F7000A296ECE00C942A2E8230E8F4E82FF0E0C0
:104F8000EE0FFF1FED52FA4F71836083813041F0C5
:104F9000809169008C7F842B80936900E89A089542
:104FA00080916900440F551F440F551F837F842B48
:104FB00080936900E99A08951F920F920FB60F929D
:104FC00011242F933F934F935F936F937F938F930E
:104FD0009F93AF93BF93EF93FF938091D3059091ED
:104FE000D405892B29F0E091D305F091D4050995DA
:104FF000FF91EF91BF91AF919F918F917F916F91B1
:105000005F914F913F912F910F900FBE0F901F9086
:1050100018951F920F920FB60F9211242F933F9362
:105020004F935F936F937F938F939F93AF93BF93B0
:10503000EF93FF938091D5059091D605892B29F0A8
:10504000E091D505F091D6050995FF91EF91BF91BB
:10505000AF919F918F917F916F915F914F913F9110
:105060002F910F900FBE0F901F9018951F920F92C7
:105070000FB60F9211242F933F938F939F93AF936B
:10508000BF938091D8059091D905A091DA05B09190
:10509000DB053091D70523E0230F2D3720F401964F
:1050A000A11DB11D05C026E8230F0296A11DB11D4B
:1050B0002093D7058093D8059093D905A093DA055E
:1050C000B093DB058091DC059091DD05A091DE05B4
:1050D000B091DF050196A11DB11D8093DC05909371
:1050E000DD05A093DE05B093DF05BF91AF919F91E1
:1050F0008F913F912F910F900FBE0F901F90189599
:105100002FB7F8946091D8057091D9058091DA0590
:105110009091DB052FBF08953FB7F8948091DC058F
:105120009091DD05A091DE05B091DF0526B5A89B25
:1051300005C02F3F19F00196A11DB11D3FBF662785
:10514000782F892F9A2F620F711D811D911D42E0CA
:10515000660F771F881F991F4A95D1F70895CF9240
:10516000DF92EF92FF92CF93DF936B017C010E945D
:105170008C28EB01C114D104E104F10479F00E9400
:105180008C286C1B7D0B683E7340A0F381E0C81A2D
:10519000D108E108F108C851DC4FECCFDF91CF9185
:1051A000FF90EF90DF90CF900895789484B582605F
:1051B00084BD84B5816084BD85B5826085BD85B5BB
:1051C000816085BDEEE6F0E0808181608083E1E86A
:1051D000F0E01082808182608083808181608083A2
:1051E000E0E8F0E0808181608083E1EBF0E08081A5
:1051F00084608083E0EBF0E0808181608083EAE777
:10520000F0E08081846080838081826080838081FF
:10521000816080838081806880831092C1000895BE
:10522000833081F028F4813099F08230A1F0089524
:105230008630A9F08730B9F08430D1F480918000B5
:105240008F7D03C0809180008F77809380000895C8
:1052500084B58F7702C084B58F7D84BD0895809119
:10526000B0008F7703C08091B0008F7D8093B00035
:105270000895CF93DF9390E0FC01ED50F44F24911B
:10528000FC01E95FF34F8491882349F190E0880F96
:10529000991FFC01E15DF34FA591B4918B5D934F94
:1052A000FC01C591D4919FB7611108C0F8948C910D
:1052B000209582238C93888182230AC0623051F426
:1052C000F8948C91322F309583238C938881822B94
:1052D000888304C0F8948C91822B8C939FBFDF91BC
:1052E000CF910895A1E0B0E0E8E7F9E20C94162E22
:1052F000282F30E0F901E152F44F8491F901ED508B
:10530000F44F1491F901E95FF34F04910023C9F0C0
:10531000882321F069830E9410296981E02FF0E041
:10532000EE0FFF1FEB5DF34FA591B4919FB7F8947B
:105330008C91611103C01095812301C0812B8C9346
:105340009FBF2196E4E00C94322ECF93DF93282F59
:1053500030E0F901E152F44F8491F901ED50F44F3E
:10536000D491F901E95FF34FC491CC2391F08111FD
:105370000E941029EC2FF0E0EE0FFF1FE55EF34FC7
:10538000A591B4912C912D2381E090E021F480E04F
:1053900002C080E090E0DF91CF910895A0E0B0E0FE
:1053A000E4EDF9E20C94122E6C017A01EB01E60EA9
:1053B000F71E00E010E0CE15DF0561F06991D6011F
:1053C000ED91FC910190F081E02DC6010995080F47
:1053D000191FF1CFC801CDB7DEB7E8E00C942E2E2F
:1053E0006115710589F0DB010D900020E9F7AD0131
:1053F00041505109461B570BDC01ED91FC91028095
:10540000F381E02D0995089580E090E00895EF92F2
:10541000FF920F931F93CF93DF938C01FB01C0E0AA
:10542000D0E064917F018FEFE81AF80A662361F0FB
:10543000D801ED91FC910190F081E02DC801099512
:10544000C80FD91FF701EDCFCE01CDB7DEB7E6E02B
:105450000C94302E0E94F0290895DC01ED91FC910E
:105460000190F081E02D099508950F931F93CF933C
:10547000DF93EC016DE00E942D2A8C016AE0CE01E1
:105480000E942D2A800F911FDF91CF911F910F91C4
:1054900008950F931F93CF93DF93EC010E94072A87
:1054A0008C01CE010E94352A800F911FDF91CF9190
:1054B0001F910F9108950F931F93CF93DF93EC01EA
:1054C0000E94F0298C01CE010E94352A800F911F85
:1054D000DF91CF911F910F9108950F931F93CF9359
:1054E000DF93EC010E942D2A8C01CE010E94352A07
:1054F000800F911FDF91CF911F910F910895A1E22D
:10550000B0E0E5E8FAE20C940E2E7C01C42EE52F03
:10551000CB01D22E19A221E02D1510F02AE0D22EB7
:105520008E010F5D1F4F8D2C912CA12CB12C6C2D59
:105530007E2FA50194010E94C72D8C2DD29E80192B
:105540001124015011098A3010F4805D01C0895C7A
:10555000F8018083211531054105510521F0C22E46
:10556000E32FCA01E4CFB801C7010E94F029A19638
:10557000ECE00C942A2EA0E0B0E0E1ECFAE20C940E
:10558000122EEC016A017B012115310541F4E881FD
:10559000F9810190F081E02D642F09951DC02A301A
:1055A0003105A9F477FF12C06DE20E942D2A8C010B
:1055B00044275527BA014C195D096E097F092AE075
:1055C000CE010E947F2A800F911F06C02AE0B701FA
:1055D000A601CE010E947F2ACDB7DEB7E8E00C9489
:1055E0002E2E9A01AB01662757FD6095762F0E94FB
:1055F000BB2A08950F931F93CF93DF93EC019A0179
:10560000AB01662757FD6095762F0E94BB2A8C015F
:10561000CE010E94352A800F911FDF91CF911F91FB
:105620000F9108952115310549F4DC01ED91FC91AC
:105630000190F081E02D642F099508950E947F2A42
:1056400008959A01462F50E060E070E00E94122B0E
:1056500008959A01AB0160E070E00E94122B08955A
:105660000F931F93CF93DF93EC010E94122B8C01B9
:10567000CE010E94352A800F911FDF91CF911F919B
:105680000F9108950F931F93CF93DF93EC019A012D
:10569000AB0160E070E00E94122B8C01CE010E94F1
:1056A000352A800F911FDF91CF911F910F9108959F
:1056B0000F931F93CF93DF93EC019A01462F50E095
:1056C00060E070E00E94122B8C01CE010E94352A0E
:1056D000800F911FDF91CF911F910F910895FC01D1
:1056E00024853585F901E05CFF4F80819181F901C6
:1056F000EE5BFF4F20813181821B930B8F739927C3
:105700000895FC0184859585FC01E05CFF4F408194
:105710005181FC01EE5BFF4F20813181421753071D
:1057200041F00190F081E02DE80FF91F808190E0B9
:1057300008958FEF9FEF0895FC0184859585FC0106
:10574000E05CFF4F40815181FC01EE5BFF4F208107
:1057500031814217530779F0A081B181A80FB91F99
:105760008C91208131812F5F3F4F2F7333273183FD
:10577000208390E008958FEF9FEF0895FC0181A1B1
:10578000882329F0A489B5898C9186FFFBCF11A2CB
:105790000895CF93DF93FC0126853785D901A05C5E
:1057A000BF4F8D919C91119701968F739927E901B5
:1057B000CE5BDF4F4881598184179507D9F30D904F
:1057C000BC91A02DA20FB31F6C93A685B785A05CDA
:1057D000BF4F11969C938E93A689B7892C9181E037
:1057E00090E0078C02C0880F991F0A94E2F7282BDB
:1057F0002C9381E081A30488F589E02D8081806469
:10580000808381E090E0DF91CF91089508951F9209
:105810000F920FB60F9211242F933F934F938F93B4
:105820009F93EF93FF938091C00082FD1CC0409135
:10583000C600809186069091870601968F739927FE
:1058400020918806309189068217930771F0E091C4
:105850008606F0918706EA5BF94F408390938706AE
:105860008093860602C08091C600FF91EF919F91C0
:105870008F914F913F912F910F900FBE0F901F90DE
:10588000189580EE95E00E946F2B892B11F00E94F5
:10589000062C08951F920F920FB60F9211242F938A
:1058A0003F938F939F93EF93FF9320914206309104
:1058B000430680914406909145062817390731F434
:1058C0008091C1008F7D8093C10014C0E091440697
:1058D000F0914506EE5FF94F20818091440690914A
:1058E000450601968F739927909345068093440649
:1058F0002093C600FF91EF919F918F913F912F913F
:105900000F900FBE0F901F901895A0E0B0E0EBE84D
:10591000FCE20C940E2EFC011382128288EE93E0BE
:10592000A0E0B0E084839583A683B7838BEB93E0FC
:10593000918380837587648757874687318B208B57
:10594000138B028BF58AE48AD78AC68AB18EA08E21
:10595000938E828E8F85848F8889858F8989868FA3
:105960008A89878F8B8980A3ECE00C942A2ECF92B2
:10597000DF92EF92FF92CF93DF93EC016A017B01FC
:10598000411581EE580761057105F9F0EC89FD8933
:1059900081E090E008A002C0880F991F0A94E2F706
:1059A000808360E079E08DE390E0A70196010E949A
:1059B000C72D215031094109510956954795379511
:1059C0002795211580E1380798F0EC89FD89108230
:1059D00060E874E88EE190E0A70196010E94C72D6F
:1059E0002150310941095109569547953795279519
:1059F000E889F9893083EA89FB89208319A2EE8935
:105A0000FF89408181E090E09C010C8C02C0220F54
:105A1000331F0A94E2F7422B4083EE89FF894081CD
:105A20009C010D8C02C0220F331F0A94E2F7422B17
:105A30004083EE89FF8940819C010E8C02C0220FB9
:105A4000331F0A94E2F7422B4083EE89FF892081BD
:105A50000F8C02C0880F991F0A94E2F78095822369
:105A60008083DF91CF91FF90EF90DF90CF900895EA
:105A70008F929F92AF92BF92CF92DF92EF92FF925E
:105A80000F931F9381E08F9385E08F9387E08F932F
:105A900083E08F9384E08F93E6EC8E2E912CF2ECD2
:105AA000AF2EB12CA1ECCA2ED12CB0ECEB2EF12CE8
:105AB00004EC10E025EC30E042E056E066E476E0ED
:105AC00080EE95E00E94852C0F900F900F900F9024
:105AD0000F901F910F91FF90EF90DF90CF90BF90AC
:105AE000AF909F908F9008950E94D5280E944522E4
:105AF000C1E4DCE20E94E1242097E1F30E94412C02
:105B0000F9CFA29FB001B39FC001A39F700D811D6B
:105B10001124911DB29F700D811D1124911D0895B6
:105B20000E94812DA59F900DB49F900DA49F800D84
:105B3000911D11240895B7FF0C94902D0E94902D73
:105B4000821B930B0895DB018F939F930E94902DEE
:105B5000BF91AF91A29F800D911DA39F900DB29F09
:105B6000900D1124089597FB072E16F4009407D08A
:105B700077FD09D00E94452E07FC05D03EF4909594
:105B800081959F4F0895709561957F4F0895A1E28B
:105B90001A2EAA1BBB1BFD010DC0AA1FBB1FEE1FA7
:105BA000FF1FA217B307E407F50720F0A21BB30BF2
:105BB000E40BF50B661F771F881F991F1A9469F76E
:105BC00060957095809590959B01AC01BD01CF01CA
:105BD0000895052E97FB1EF400940E94002E57FD99
:105BE00007D00E94C72D07FC03D04EF40C94002E62
:105BF00050954095309521953F4F4F4F5F4F0895F9
:105C000090958095709561957F4F8F4F9F4F089528
:105C10002F923F924F925F926F927F928F929F92BC
:105C2000AF92BF92CF92DF92EF92FF920F931F93AA
:105C3000CF93DF93CDB7DEB7CA1BDB0B0FB6F8945B
:105C4000DEBF0FBECDBF09942A88398848885F849B
:105C50006E847D848C849B84AA84B984C884DF800C
:105C6000EE80FD800C811B81AA81B981CE0FD11DF0
:105C70000FB6F894DEBF0FBECDBFED010895EE0F55
:105C8000FF1F0590F491E02D0994AA1BBB1B51E165
:105C900007C0AA1FBB1FA617B70710F0A61BB70B9C
:105CA000881F991F5A95A9F780959095BC01CD0141
:105CB00008958F929F92AF92BF92CF92DF92EF9210
:105CC000FF92CF93DF93EC01688179818A819B8178
:105CD000611571058105910521F464E279ED8BE58B
:105CE00097E02DE133EF41E050E00E94E92D4901BA
:105CF0005A019B01AC01A7EAB1E40E94902D6B010F
:105D00007C01ACEEB4EFA50194010E949E2DC60E5D
:105D1000D71EE81EF91EF7FE06C081E0C81AD1089A
:105D2000E10880E8F80AC882D982EA82FB82C701CA
:105D3000B6019F77DF91CF91FF90EF90DF90CF90EA
:105D4000BF90AF909F908F9008950E94592E089514
:105D500086E091E00E94592E0895609306017093A9
:105D60000701809308019093090108952F923F92B3
:105D70005F926F927F928F929F92AF92BF92CF92DB
:105D8000DF92EF92FF920F931F93CF93DF938B01DC
:105D9000EA016115710521F0DB018C9311969C934A
:105DA000209739F09E01225031092332310508F045
:105DB000D8C07C016701BFEFCB1ADB0A5601F7019F
:105DC0006080862D90E00E94E82F892B11F07601EB
:105DD000F1CFFDE26F120AC0570182E0A80EB11C9C
:105DE000D70111966C90772473940BC0BBE26B12B1
:105DF00007C05701E2E0AE0EB11CD70111966C90BE
:105E0000712CCE018F7E892B89F4B0E36B1237C0E1
:105E1000F50180818F7D8835D1F46180F2E0AF0E8D
:105E2000B11C872D8260782EC0E1D0E0CA30D10548
:105E300051F1C031D10521F0C830D10599F409C024
:105E4000CC24CA94DC2CEC2CAFE0FA2E22C0209794
:105E500069F7C8E0D0E0CC24CA94DC2CEC2CFFE13C
:105E6000FF2E17C06FEF7FEFCB019E01442737FD58
:105E70004095542F0E94C72D69017A010AC02097CE
:105E8000A9F6CAE0D0E0E9E9CE2EDC2CEC2CE9E161
:105E9000FE2EF50160E020E030E0A9014E01AA24C9
:105EA00097FCA094BA2C1F0170ED572E560CA9E058
:105EB000A51570F48FEB860D8A3118F499EC592EE4
:105EC00006C08FE9860D8A3148F589EA582E560CAE
:105ED000852D90E08C179D070CF56F3FD9F0C21609
:105EE000D306E406F50698F0C501B4010E94A32D7F
:105EF0009B01AC01852D90E0A0E0B0E0280F391F98
:105F00004A1F5B1F281739074A075B0710F46FEF1A
:105F100001C061E03196D1016C90C5CF011511052A
:105F200051F0662311F0319703C071FE04C032971F
:105F3000D801ED93FC9370FE07C0509540953095C5
:105F400021953F4F4F4F5F4F67FF10C082E290E0B7
:105F500090938B0680938A066FEF7FEF8FEF9FEF12
:105F600007C060E070E080E090E002C0B901CA01C3
:105F7000DF91CF911F910F91FF90EF90DF90CF9025
:105F8000BF90AF909F908F907F906F905F903F9069
:105F90002F900895FC0188279927E89421912032B9
:105FA000E9F3293010F02E30C8F32B3241F02D32B6
:105FB00039F4689404C00E941C30820F911D219115
:105FC00020532A30C0F31EF4909581959F4F089579
:105FD000911150C0803219F089508550D0F7089542
:105FE00048EC53E00E94F52F0895FA01A191B08189
:105FF000009719F41097E1F0CD01DC01CD010D906F
:10600000002011F4C00113C0FB012191222319F0DB
:106010002015D9F7F3CFFB012191201519F41E9219
:10602000119606C02223C1F70D900020A1F7D001E0
:10603000FA01A193B08308957AE0979F902D879FEE
:10604000802D910D11240895F999FECF92BD81BD47
:10605000F89A992780B50895262FF999FECF1FBA8F
:1060600092BD81BD20BD0FB6F894FA9AF99A0FBE81
:0E60700001960895992788270895F894FFCF88
:10607E0000008C06200001000000FF00020002005C
:10608E0002000200020002000200020002000200F2
:10609E00020002000200020002000280250000053C
:1060AE00400AA1204EA50020244EA52C2330C0125C
:1060BE0000001A400AA1204EA5001B1E27522C23B9
:1060CE00308025000005400AA1204EA50020244E58
:1060DE00A52C2330004B000006400AD0009D49003D
:1060EE007B289D492C233000E1000005400A450124
:1060FE00D7DC03B81E0EBF00232E48E801008A40ED
:10610E000A6001555502AD1E20000023C8545820C8
:10611E0074696D656F75742100596573004E6F005B
:10612E002C00386368004E2F41002C205B005D2050
:10613E0028002900486F70206368616E6E656C20C0
:10614E000020402000456E746572696E67206164A0
:10615E00617074697665206368616E6E656C20731C
:10616E00656C656374696F6E2C207069636B696E04
:10617E00673A007363616E6E6572206D6F646500C1
:10618E004E4F5420454E41424C45440053656E647B
:10619E00696E672073657474696E677320746F20FF
:1061AE0052580A00526573657474696E6720736580
:1061BE007474696E6773206F6E2052580A004162C4
:1061CE006F727465642065646974730A00696E7613
:1061DE00616C69642073656C656374696F6E000D24
:1061EE000A496E76616C696420696E707574202D33
:1061FE00206469736361726465642107005365747A
:10620E0074696E677320736176656420746F2045C0
:10621E004550524F4D0A0052657665727465642082
:10622E0073657474696E67732066726F6D20454571
:10623E0050524F4D0A004C6F616465642066616375
:10624E00746F72792064656661756C74730A004BA5
:10625E00657920616E64206368616E6E656C732073
:10626E0072616E646F6D697A65640A004F70656E57
:10627E004C52536E67205458207374617274696E59
:10628E00672000206F6E20485720006D6F64756C7C
:10629E0065206C6F636B65643F00342B34003800EF
:1062AE00382B340031320031322B3400313600506D
:1062BE00504D0052535349005344410053434C0038
:1062CE00525844005458440041494E004C424545F2
:1062DE00500053504B54524D00534255530053559A
:1062EE004D44004C4C494E440000070B0C10111548
:1062FE0000B6012A032E033003340337033C03B6E2
:10630E00013F03430348034C035003540358035CFB
:10631E0003620369036E0373038C028C028C028C7E
:10632E0002160A1322312900000000C92BCE296F54
:08633E002B9C2B812BBE2B00D0
:107E00000F92CDB7DEB7112484B714BE81FFF1D035
:107E100082E08093C00088E18093C10086E0809377
:107E2000C20080E18093C4008EE0CDD088249924E4
:107E3000CC24C394F5E0DF2EE1E1EE2E73E0F72EC3
:107E4000B6D0082F813479F4B2D08983C2D0898129
:107E5000823811F481E005C0813811F485E001C059
:107E600083E09ED09AC0823411F484E103C085344B
:107E700019F485E0B6D091C0853561F498D0082F0B
:107E800010E095D090E0982E8824802A912A880CC2
:107E9000991C82C0863521F484E0A3D080E0E1CF34
:107EA000843609F04CC083D082D0A82E80D0B82E62
:107EB00000E011E07CD0F80181938F01AE16D1F77C
:107EC00088D0FB2DF53489F4E0E0F1E00BC0F9999E
:107ED000FECF92BC81BC0894811C911C819180BD15
:107EE000FA9AF99AEA1598F358C08B2D863409F05E
:107EF00054C0F401F7BEE89507B600FCFDCFF401CD
:107F0000A0E0B1E02C9130E011968C91119790E0B7
:107F1000982F8827822B932B12960C01C7BEE895C9
:107F20001124329681E0A038B80761F7F401D7BE7A
:107F3000E89507B600FCFDCFE7BEE8952EC0843774
:107F4000F1F435D034D0182F32D0B82E42D0FB2DDA
:107F5000F63421F4F40105914F010CC0FB2DF534EA
:107F600049F4F999FECF92BC81BC0894811C911C04
:107F7000F89A00B5802F14D0115049F70EC08537FC
:107F800039F427D08EE10CD085E90AD08FE069CF93
:107F9000813511F488E017D01CD080E101D050CF9A
:107FA0009091C00095FFFCCF8093C600089580910A
:107FB000C00087FFFCCF8091C00084FD01C0A89560
:107FC0008091C6000895E0E6F0E098E19083808318
:107FD0000895EDDF803219F088E0F5DFFFCF84E10E
:107FE000DFCF1F93182FE3DF1150E9F7F2DF1F9166
:0E7FF0000895282E80E0E7DFEE27FF27099492
:027FFE0001057B
:0400000300007E007B
:00000001FF
